:02000000502886
:1000080009008A0132088207CF28F7288F28B028EC
:10001800D728082923088A01A0000310A00D20086A
:1000280082078716080007160800051408008514BB
:10003800080005150800071408000715080006162B
:100048000800861608000617080087170800861794
:1000580008008716080023088A01A0000310A00DD5
:1000680020088207871208000712080005100800F8
:10007800851008000511080007100800071108007E
:1000880006120800861208000613080087130800E5
:100098008613080087120800831600308500003098
:1000A80086004830870020309F0070308F00831210
:1000B800031780309E0001309F0003132D14AE15E6
:1000C8008710B2010F30B300850186018701051240
:1000D80023217E210730942185165D21A100143C3F
:1000E80003187B282108FF3A031983286B28051673
:1000F8005921B03C031C6B28832188206B2885126A
:1001080087149B2187106B280520B20A3208053C0A
:10011800031CB20108004030AC009520AC0B9128BC
:10012800080000309C2001309C2002309C200800F0
:10013800A3000430B1000E200330A307B10B9F28A1
:100148002C0894212C0894212C0894212C08942103
:100158002C089421232108000530B4002B210030FD
:10016800B1000130B00023080F202308013E3020E1
:1001780030083106031DC528230830202308013E16
:100188000F20B00FBC28B10BB528A30AA20BB328C7
:10019800B40BB22808005030AC00F2202C088E2195
:1001A800AC0BD12808000A30B4002B2123080F20FB
:1001B80034088E21A30AA20BDA282B212308302029
:1001C80034088E21A30AA20BE228F22001308821EC
:1001D800F2200A308821B40BD9280800871414307B
:1001E8009421871008000F30B4000C30A200A3013E
:1001F80023080F2034088E2123083020A30AA20BDD
:10020800FC28B40BF9280800FA30B4000330A20027
:100218004E210F39A3000C3C031C0C2923080F2086
:100228001430942123083020A20B0C29B40B0A297E
:1002380008002321023088210F30B30008002B2149
:1002480023083020A30AA20B2429871008000C30A9
:10025800A200A30108004E213F39143EAC0008005B
:100268002C089429193094218501860187010800FA
:10027800051685160A3094215921A8215D21A82147
:1002880085120A3094215921A8215D21A821143012
:1002980088213C292D08AE072E08AF070310AF0CA4
:1002A8000318AF172F08AD07080008306821240885
:1002B800080007306021080068210310A50CA40C71
:1002C800A50CA40C240808000F39A0000310A00DE9
:1002D800A00D813020049F009B219F140000000086
:1002E8009F18742983161E088312A4001E08A500EF
:1002F8009F100800831601308F00831208008316B0
:1003080071308F0083120800AB0064309421AB0B6E
:1003180089290800AB000A309421AB0B8F2908000B
:10032800AA009D21AA0B9529080002309E291430A5
:100338009E29C830A900000000000000000000004D
:100348000000A90B9F290800AB21C8309429B500EB
:100358000830B6000514C421C421C4210510C421E5
:100368000514C421B50D0318C4210510C421031CAC
:10037800C421B60BB4290514C4210510C421C42115
:0A0388000830B700B70BC6290800C3
:02400E00E400CC
:00000001FF
